:100000000C943A010C946B010C946B010C946B01F1
:100010000C946B010C946B010C946B010C946B01B0
:100020000C946B010C946B010C946B010C946B01A0
:100030000C946B010C946B010C946B010C946B0190
:100040000C946B010C94F5060C946B010C946B01F1
:100050000C946B010C946B010C946B010C940E09C5
:100060000C946B010C94770B0C94670C0C946B0143
:100070000C946B010C946B010C946B010C946B0150
:100080000C9423070C946B010C946B010C946B0182
:100090000C94AB0B0C94A60C0C946B010C946B01A0
:1000A0000C946B010C946B010C9451070C946B0134
:1000B0000C946B010C946B010C946B010C947F07F6
:1000C0000C946B010C946B010C946B010C94DF0B82
:1000D0000C94E50C0C946B010C94130C0C94240DF3
:1000E0000C946B011C0A1F0A120A160A560A230AEC
:1000F000270A2D0A310A350A3B0A3F0A430A560AE3
:10010000490A4D0A510A0C94350A0C941C0A0C94A5
:10011000430A0C941F0A0C942D0A0C940F0B0C9498
:10012000EB0D0C941A0B0C94120A0C94D30A0C9439
:10013000EF0A0C94310A0C94560A0C94510A0C9450
:10014000160A0C94230A0C94460C0C94270A0C945F
:10015000C30A0C94490A0C943F0A0C940B0F0C949C
:100160002A060C944D0A0C943B0A0000090A020866
:100170000B0C0D0706030401000000000000000046
:10018000000000000000000000000000000000006F
:1001900000000000000011100F000000000000002F
:1001A000000000000000000000000000000000004F
:1001B0000102102020080810204010204080020179
:1001C000020108040201010204081020408080405E
:1001D000201008040201800402018040201008045D
:1001E00002010804020101020408102040800102FB
:1001F00004081020408005050505070508080808C3
:10020000020202020A0A08080404040401010101AE
:1002100001010101030303030303030304070707A9
:100220000C0C0C0C0C0C0C0C02020202060606064E
:10023000060606060B0B0B0B0B0B0B0B000022002C
:10024000250028002B002E003100340002010000A0
:10025000050108010B0100002100240027002A00ED
:100260002D003000330001010000040107010A01E4
:100270002A06EB0D11241FBECFEFD1E2DEBFCDBFAA
:1002800000E00CBF12E0A0E0B2E0ECEEFFE100E025
:100290000BBF02C007900D92A43BB107D9F725E030
:1002A000A4EBB2E001C01D92AF3FB207E1F711E04D
:1002B000CAE3D1E000E006C021970109802FFE01CA
:1002C0000E94D20FC833D10780E00807A9F70E9427
:1002D000BD0E0C94F40F0C94000040E855E260E071
:1002E00070E08DEB93E00E94630D61E083E00E947B
:1002F000570A61E084E00E94570A61E085E00E94AD
:10030000570A61E086E00E94570A61E087E00E9498
:10031000570A61E088E00E94570A61E089E00E9484
:10032000570A61E08AE00E94570A61E08BE00E9470
:10033000570A61E08CE00E94570A61E08DE00E945C
:10034000570A66E070E086EB92E00E94770861E071
:10035000809100020C94570ACF93DF9362E072E021
:100360008DEB93E00E94630F61E08DE00E94930AA1
:100370006CE271E080E090E00E947D0960E08DE039
:100380000E94930A6CE271E080E090E00E947D0997
:1003900061E08CE00E94930A6CE271E080E090E002
:1003A0000E947D0960E08CE00E94930A6CE271E09B
:1003B00080E090E00E947D0961E08DE00E94930A58
:1003C0006CE271E080E090E00E947D0960E08DE0E9
:1003D0000E94930A6CE271E080E090E00E947D0947
:1003E00061E08CE00E94930A6CE271E080E090E0B2
:1003F0000E947D0960E08CE00E94930A6CE271E04B
:1004000080E090E00E947D0961E08DE00E94930A07
:1004100061E08CE00E94930A64EF71E080E090E07C
:100420000E947D0960E08DE00E94930A60E08CE00C
:100430000E94930A64EF71E080E090E00E947D09E1
:1004400061E084E00E94930A6CE271E080E090E059
:100450000E947D0960E084E00E94930A6CE271E0F2
:1004600080E090E00E947D0961E084E00E94930AB0
:100470006CE271E080E090E00E947D0960E084E041
:100480000E94930A6CE271E080E090E00E947D0996
:1004900061E084E00E94930A6CE271E080E090E009
:1004A0000E947D0960E084E00E94930A6CE271E0A2
:1004B00080E090E00E947D0961E08DE00E94930A57
:1004C00061E08CE00E94930A64EF71E080E090E0CC
:1004D0000E947D0960E08DE00E94930A60E08CE05C
:1004E0000E94930A64EF71E080E090E00E947D0931
:1004F00061E08DE00E94930A6CE271E080E090E0A0
:100500000E947D0960E08DE00E94930A6CE271E038
:1005100080E090E00E947D0961E08CE00E94930AF7
:100520006CE271E080E090E00E947D0960E08CE088
:100530000E94930A6CE271E080E090E00E947D09E5
:1005400061E08DE00E94930A6CE271E080E090E04F
:100550000E947D0960E08DE00E94930A6CE271E0E8
:1005600080E090E00E947D0961E08CE00E94930AA7
:100570006CE271E080E090E00E947D0960E08CE038
:100580000E94930A6CE271E080E090E00E947D0995
:1005900061E08DE00E94930A61E08CE00E94930A82
:1005A00064EF71E080E090E00E947D0960E08DE002
:1005B0000E94930A60E08CE00E94930A64EF71E06D
:1005C00080E090E00E947D0961E08DE00E94930A46
:1005D00061E08CE00E94930A64EF71E080E090E0BB
:1005E0000E947D0960E08DE00E94930A60E08CE04B
:1005F0000E94930A64EF71E080E090E00E947D0920
:1006000061E084E00E94930A6CE271E080E090E097
:100610000E947D0960E084E00E94930A6CE271E030
:1006200080E090E00E947D0961E084E00E94930AEE
:100630006CE271E080E090E00E947D0960E084E07F
:100640000E94930A6CE271E080E090E00E947D09D4
:1006500061E084E00E94930A6CE271E080E090E047
:100660000E947D0960E084E00E94930A6CE271E0E0
:1006700080E090E00E947D0965E172E08DEB93E0FF
:100680000E94630F61E08BE00E94930A68EE73E0C2
:1006900080E090E00E947D0960E08BE00E94930A78
:1006A00068EE73E080E090E00E947D0961E08AE0FE
:1006B0000E94930A68EE73E080E090E00E947D095A
:1006C00060E08AE00E94930A68EE73E080E090E0C8
:1006D0000E947D0961E089E00E94930A68EE73E060
:1006E00080E090E00E947D0960E089E00E94930A2A
:1006F00068EE73E080E090E00E947D0960E372E0C4
:100700008DEB93E00E94630F61E088E00E94930A02
:1007100068EE73E080E090E00E947D0960E088E090
:100720000E94930A68EE73E080E090E00E947D09E9
:1007300061E087E00E94930A68EE73E080E090E059
:100740000E947D0960E087E00E94930A68EE73E0F2
:1007500080E090E00E947D0961E087E00E94930ABA
:1007600068EC70E080E090E00E947D0960E087E046
:100770000E94930A68EC70E080E090E00E947D099E
:1007800061E087E00E94930A68EC70E080E090E00E
:100790000E947D0960E087E00E94930A68EC70E0A7
:1007A00080E090E00E947D0961E087E00E94930A6A
:1007B00068EC70E080E090E00E947D0960E087E0F6
:1007C0000E94930A68EC70E080E090E00E947D094E
:1007D00061E087E00E94930A68EC70E080E090E0BE
:1007E0000E947D0960E087E00E94930A6CE271E05C
:1007F00080E090E00E947D0965E172E08DEB93E07E
:100800000E94630F61E08BE00E94930A68EE73E040
:1008100080E090E00E947D0960E08BE00E94930AF6
:1008200068EE73E080E090E00E947D0961E08AE07C
:100830000E94930A68EE73E080E090E00E947D09D8
:1008400060E08AE00E94930A68EE73E080E090E046
:100850000E947D0961E089E00E94930A68EE73E0DE
:1008600080E090E00E947D0960E089E00E94930AA8
:1008700068EE73E080E090E00E947D0960E372E042
:100880008DEB93E00E94630F61E088E00E94930A81
:1008900068EE73E080E090E00E947D0960E088E00F
:1008A0000E94930A68EE73E080E090E00E947D0968
:1008B00061E087E00E94930A68EE73E080E090E0D8
:1008C0000E947D0960E087E00E94930A68EE73E071
:1008D00080E090E00E947D0961E087E00E94930A39
:1008E00068EC70E080E090E00E947D0960E087E0C5
:1008F0000E94930A68EC70E080E090E00E947D091D
:1009000061E087E00E94930A68EC70E080E090E08C
:100910000E947D0960E087E00E94930A68EC70E025
:1009200080E090E00E947D0961E087E00E94930AE8
:1009300068EC70E080E090E00E947D0960E087E074
:100940000E94930A68EC70E080E090E00E947D09CC
:1009500061E087E00E94930A68EC70E080E090E03C
:100960000E947D0960E087E00E94930A6CE271E0DA
:1009700080E090E00E947D096EE472E08DEB93E0F0
:100980000E94630FC3E0D0E061E0809100020E940A
:10099000930A61E672E08DEB93E00E94630F64E6D8
:1009A00070E080E090E00E947D0960E080910002AC
:1009B0000E94930A60E772E08DEB93E00E94630F60
:1009C00064E670E080E090E00E947D0961E0809143
:1009D00000020E94930A61E672E08DEB93E00E94B0
:1009E000630F64E670E080E090E00E947D0960E0C3
:1009F000809100020E94930A60E772E08DEB93E021
:100A00000E94630F64E670E080E090E00E947D0940
:100A100061E0809100020E94930A61E672E08DEB32
:100A200093E00E94630F64E670E080E090E00E9433
:100A30007D0960E0809100020E94930A60E772E005
:100A40008DEB93E00E94630F64E670E080E090E03D
:100A50000E947D09219709F097CF6EE772E08DEB38
:100A600093E00E94630F64E670E080E090E00E94F3
:100A70007D0962E972E08DEB93E00E94630F82E3EF
:100A800090E09093B5028093B4026091B4027091AB
:100A9000B5026937710584F486EB92E00E94B208D2
:100AA00062E370E080E090E00E947D098091B402F2
:100AB0009091B5020196E5CF88E790E09093B5025A
:100AC0008093B4026091B4027091B50262337105F3
:100AD00084F086EB92E00E94B20862E370E080E06E
:100AE00090E00E947D098091B4029091B502019737
:100AF000E5CF8EE190E09093B5028093B4026091CF
:100B0000B4027091B5026739710584F486EB92E006
:100B10000E94B20862E370E080E090E00E947D09EC
:100B20008091B4029091B5020196E5CF86E990E0FC
:100B30009093B5028093B4026091B4027091B502B3
:100B40006E31710584F086EB92E00E94B20862E398
:100B500070E080E090E00E947D098091B402909165
:100B6000B5020197E5CF82E390E09093B5028093C0
:100B7000B4026091B4027091B5026937710584F4D2
:100B800086EB92E00E94B20862E370E080E090E0C1
:100B90000E947D098091B4029091B5020196E5CF43
:100BA00088E790E09093B5028093B4026091B4021C
:100BB0007091B5026233710584F086EB92E00E9479
:100BC000B20862E370E080E090E00E947D098091CD
:100BD000B4029091B5020197E5CF84E690E090933E
:100BE000B5028093B4026091B4027091B502673986
:100BF000710584F486EB92E00E94B20862E370E033
:100C000080E090E00E947D098091B4029091B5024D
:100C10000196E5CF86E990E09093B5028093B40207
:100C20006091B4027091B5026436710584F086EB70
:100C300092E00E94B20862E370E080E090E00E94DF
:100C40007D098091B4029091B5020197E5CFDF91C3
:100C5000CF91089586EB92E00C94AD07CF92DF928E
:100C6000EF92FF920F931F93CF93DF936C018B0151
:100C70007A01EC01C654DD4F888187FF04C0FB0177
:100C80001182108224C08CE08C9D90018D9D300DCE
:100C900011248881A901480F511D87FD5A95809123
:100CA000B90290E04817590794F48881A901480FC8
:100CB000511D87FD5A95CA01FA01EE0FFF1F8E0FD5
:100CC0009F1FFC01E254FD4F808186FD19C0888181
:100CD0008F5F88838CE08C9D90018D9D300D112459
:100CE0008881A901480F511D87FD5A958091B9024D
:100CF00090E048175907BCF488818C3044F113C048
:100D00008881280F311D87FD3A95F901EE0FFF1FED
:100D10002E0F3F1FF901E254FD4F808160E08F7379
:100D20000E94930AD4CFF801808191810496803487
:100D30009C4918F480E49CE904C0F8018081918109
:100D40000496F701918380838FEF888345C0F80173
:100D5000408151818881B901680F711D87FD7A95A5
:100D6000CB01FB01EE0FFF1F8E0F9F1FFC01E25412
:100D7000FD4F81819281840F951FF70191838083BC
:100D80008881A901480F511D87FD5A95CA01FA01B2
:100D9000EE0FFF1F8E0F9F1FFC01E254FD4F80815D
:100DA00086FF1AC08881280F311D87FD3A95F90109
:100DB000EE0FFF1F2E0F3F1FF901E254FD4F808100
:100DC00061E08F73DF91CF911F910F91FF90EF90B2
:100DD000DF90CF900C94930ADF91CF911F910F91E8
:100DE000FF90EF90DF90CF9008951F920F920FB673
:100DF0000F9211240BB60F922F933F934F935F9353
:100E00006F937F938F939F93AF93BF93EF93FF93D2
:100E100048E850E064E870E081E090E00E942E062F
:100E2000FF91EF91BF91AF919F918F917F916F91C2
:100E30005F914F913F912F910F900BBE0F900FBE7E
:100E40000F901F9018951F920F920FB60F921124BA
:100E50000BB60F922F933F934F935F936F937F93B4
:100E60008F939F93AF93BF93EF93FF9348E950E025
:100E700064E970E082E090E00E942E06FF91EF911D
:100E8000BF91AF919F918F917F916F915F914F91A2
:100E90003F912F910F900BBE0F900FBE0F901F90A0
:100EA00018951F920F920FB60F9211240BB60F9246
:100EB0002F933F934F935F936F937F938F939F9362
:100EC000AF93BF93EF93FF9348EA50E064EA70E07A
:100ED00083E090E00E942E06FF91EF91BF91AF91C9
:100EE0009F918F917F916F915F914F913F912F9142
:100EF0000F900BBE0F900FBE0F901F9018951F9272
:100F00000F920FB60F9211240BB60F922F933F93AF
:100F10004F935F936F937F938F939F93AF93BF9301
:100F2000EF93FF9348E251E064E271E080E090E0EB
:100F30000E942E06FF91EF91BF91AF919F918F91EB
:100F40007F916F915F914F913F912F910F900BBEC9
:100F50000F900FBE0F901F901895FC019091B90251
:100F60009033A0F481E0890F8093B9029083892F98
:100F700090E0FC01EE0FFF1F8E0F9F1FFC01E2545B
:100F8000FD4F88EB9BE09283818308958FEF8083F0
:100F90000895DF92EF92FF920F931F93CF93DF9309
:100FA000EC01D62E7A0189018881803308F06AC06D
:100FB00061E08D2D0E94570A8881E82FF0E09F01A3
:100FC000220F331FE20FF31FE254FD4F9D2D9F733D
:100FD0002081207CD22ED92AD08260E272E0AB013F
:100FE0004E195F0957FF02C04D5F5F4F55954795FA
:100FF00055954795498340E659E09A01201B310BEE
:1010000037FF02C02D5F3F4F3595279535952795C2
:101010002A836CE00E94850F9CE0899FB001112417
:1010200040E050E09A01260F371FF901EE0FFF1F35
:101030002E0F3F1FF901E254FD4F908196FD16C01F
:101040004F5F5F4F4C30510569F7813021F51092A9
:10105000800082E0809381001092850010928400CD
:10106000B19A80916F00826080936F00E881F0E018
:10107000CF01880F991FE80FF91FE254FD4F8081BF
:10108000806480838881DF91CF911F910F91FF90C1
:10109000EF90DF900895823061F410929000809379
:1010A0009100109295001092940088BB809371007B
:1010B000DDCF833069F41092A00082E08093A1001C
:1010C0001092A5001092A40089BB80937200CECF2D
:1010D0008111CCCF1092200182E0809321011092E7
:1010E0002501109224018ABB80937300BFCF20E6B4
:1010F00039E040E252E00C94C907FC019081903342
:1011000080F5818128E830E0281B310987FD33957F
:10111000220F331F220F331F621773077CF0828167
:1011200028E532E0281B310987FD3395220F331F54
:10113000220F331F621773070CF49B014FB7F8940B
:10114000892F90E0FC01EE0FFF1F8E0F9F1FFC0107
:10115000E254FD4F22503109220F331F3283218385
:101160004FBF0895AF92BF92CF92DF92EF92FF925E
:101170000F931F93CF93DF93EC01603282E07807E7
:101180000CF03FC077FD06C0653B71052CF064EBA9
:1011900070E002C060E070E0898128E830E0590129
:1011A000A81AB10887FDB394AA0CBB1CAA0CBB1CDF
:1011B0000B2C000CCC08DD08072E000C880B990BBB
:1011C0002A8108E512E0021B110927FD1395000F83
:1011D000111F000F111F012E000C220B330B3F9328
:1011E0002F931F930F9314EBE12EF12C00E010E0EE
:1011F00020E030E0A9010E94CA0E0F900F900F90DE
:101200000F90CE01DF91CF911F910F91FF90EF9042
:10121000DF90CF90BF90AF900C947D081F920F92FB
:101220000FB60F9211242F933F938F939F93AF93F9
:10123000BF9380914F0390915003A0915103B091BF
:10124000520330914E0323E0230F2D3720F40196F3
:10125000A11DB11D05C026E8230F0296A11DB11DD9
:1012600020934E0380934F0390935003A093510318
:10127000B09352038091530390915403A09155036E
:10128000B09156030196A11DB11D80935303909315
:101290005403A0935503B0935603BF91AF919F9110
:1012A0008F913F912F910F900FBE0F901F90189527
:1012B0003FB7F8948091530390915403A091550344
:1012C000B091560326B5A89B05C02F3F19F0019693
:1012D000A11DB11D3FBFBA2FA92F982F8827820FBC
:1012E000911DA11DB11DBC01CD0142E0660F771F0C
:1012F000881F991F4A95D1F70895CF92DF92EF92F8
:10130000FF92CF93DF936B017C010E945809EB01A0
:10131000C114D104E104F10479F00E9458096C1B56
:101320007D0B683E7340A0F381E0C81AD108E10844
:10133000F108C851DC4FECCFDF91CF91FF90EF90D7
:10134000DF90CF900895789484B5826084BD84B591
:10135000816084BD85B5826085BD85B5816085BDB0
:10136000EEE6F0E0808181608083E1E8F0E01082C9
:10137000808182608083808181608083E0E8F0E00A
:10138000808181608083E1EBF0E0808184608083F4
:10139000E0EBF0E0808181608083E1E9F0E0808132
:1013A00082608083808181608083E0E9F0E08081D9
:1013B00081608083E1EAF0E08081826080838081C7
:1013C00081608083E0EAF0E0808181608083E1E2F7
:1013D000F1E0808182608083808181608083E0E2AF
:1013E000F1E0808181608083EAE7F0E080818460C1
:1013F000808380818260808380818160808380811E
:10140000806880831092C100089590E0FC013197BC
:10141000E131F10508F04AC08827EE58FF4F8F4FA1
:101420000C94D20F809180008F7703C08091800050
:101430008F7D80938000089584B58F7702C084B536
:101440008F7D84BD08958091B0008F7703C0809117
:10145000B0008F7D8093B0000895809190008F77C9
:1014600007C0809190008F7D03C080919000877F9E
:101470008093900008958091A0008F7707C080919D
:10148000A0008F7D03C08091A000877F8093A00083
:101490000895809120018F7707C0809120018F7D72
:1014A00003C080912001877F809320010895CF930E
:1014B000DF9390E0FC01E055FE4F2491FC01EA50DF
:1014C000FE4F8491882361F190E0880F991FFC0101
:1014D000EA5AFD4FC591D491FC01E45CFD4FA59102
:1014E000B491611109C09FB7F89488812095822337
:1014F0008883EC912E230BC0623061F49FB7F8947F
:101500003881822F809583238883EC912E2B2C9316
:101510009FBF06C08FB7F894E8812E2B28838FBF1A
:10152000DF91CF9108951F93CF93DF93282F30E061
:10153000F901E659FE4F8491F901E055FE4FD4912F
:10154000F901EA50FE4FC491CC23C9F0162F811146
:101550000E94050AEC2FF0E0EE0FFF1FE45CFD4F48
:10156000A591B4918FB7F894111105C09C91ED2FFE
:10157000E095E92302C0EC91ED2BEC938FBFDF9156
:10158000CF911F910895FC0124853585F901E05C18
:10159000FF4F80819181329620813181821B930B94
:1015A0008F7399270895DC011C96ED91FC911D978E
:1015B000DF01A05CBF4F2D913C91119712968D9148
:1015C0009C9111972817390739F08D919C91E80F5C
:1015D000F91F808190E008958FEF9FEF0895FC013F
:1015E000A485B585FD01E05CFF4F208131813296F5
:1015F000808191812817390779F080819181A80F26
:10160000B91F8C91208131812F5F3F4F2F7333277A
:101610003183208390E008958FEF9FEF0895FC01C0
:1016200081A1882329F0A489B5898C9186FFFBCFFD
:1016300011A208950F931F93CF93DF93FC01A6850A
:10164000B7858D01005C1F4FE80188819981019663
:101650008F739927AD014E5B5F4FEA012881398175
:1016600082179307D1F3E80128813981A20FB31FB4
:101670006C93A685B785A05CBF4F11969C938E9303
:10168000A689B7892C9181E090E0078C02C0880F71
:10169000991F0A94E2F7822B8C9381E081A304883E
:1016A000F589E02D80818064808381E090E0DF9186
:1016B000CF911F910F910895FB01E05CFF4F2081B6
:1016C00031812F5F3F4F2F733327DB01AE5BBF4F5D
:1016D0004D915C912417350741F040815181DB0128
:1016E000A40FB51F8C9331832083089508951F9212
:1016F0000F920FB60F9211240BB60F922F933F93B8
:101700004F935F936F937F938F939F93AF93BF9309
:10171000EF93FF938091C00082FD07C08091C600C7
:101720006BEB75E00E945C0B02C08091C600FF91DC
:10173000EF91BF91AF919F918F917F916F915F9149
:101740004F913F912F910F900BBE0F900FBE0F90B6
:101750001F90189508951F920F920FB60F921124A3
:101760000BB60F922F933F934F935F936F937F939B
:101770008F939F93AF93BF93EF93FF938091C80094
:1017800082FD07C08091CE0063E375E00E945C0B90
:1017900002C08091CE00FF91EF91BF91AF919F91D8
:1017A0008F917F916F915F914F913F912F910F900A
:1017B0000BBE0F900FBE0F901F90189508951F92AB
:1017C0000F920FB60F9211240BB60F922F933F93E7
:1017D0004F935F936F937F938F939F93AF93BF9339
:1017E000EF93FF938091D00082FD07C08091D600D7
:1017F0006BEA74E00E945C0B02C08091D600FF91FE
:10180000EF91BF91AF919F918F917F916F915F9178
:101810004F913F912F910F900BBE0F900FBE0F90E5
:101820001F90189508951F920F920FB60F921124D2
:101830000BB60F922F933F934F935F936F937F93CA
:101840008F939F93AF93BF93EF93FF93809130015A
:1018500082FD07C08091360163E274E00E945C0B58
:1018600002C080913601FF91EF91BF91AF919F919E
:101870008F917F916F915F914F913F912F910F9039
:101880000BBE0F900FBE0F901F9018958DEB93E03D
:101890000E94C30A892B11F00E94760B8BE993E01A
:1018A0000E94C30A892B11F00E94AA0B89E793E0DA
:1018B0000E94C30A892B11F00E94DE0B87E593E09A
:1018C0000E94C30A892B11F00C94120C08951F92E8
:1018D0000F920FB60F9211240BB60F922F933F93D6
:1018E0008F939F93EF93FF932091B7053091B805A5
:1018F0008091B9059091BA052817390731F4809184
:10190000C1008F7D8093C10014C0E091B905F091B2
:10191000BA05E958FA4F20818091B9059091BA052E
:1019200001968F7399279093BA058093B9052093F8
:10193000C600FF91EF919F918F913F912F910F9052
:101940000BBE0F900FBE0F901F9018951F920F9215
:101950000FB60F9211240BB60F922F933F938F93D4
:101960009F93EF93FF9320912F0530913005809145
:101970003105909132052817390731F48091C9005B
:101980008F7D8093C90014C0E0913105F09132053C
:10199000E151FB4F208180913105909132050196F4
:1019A0008F73992790933205809331052093CE0051
:1019B000FF91EF919F918F913F912F910F900BBECF
:1019C0000F900FBE0F901F9018951F920F920FB699
:1019D0000F9211240BB60F922F933F938F939F93E7
:1019E000EF93FF932091A7043091A8048091A9045C
:1019F0009091AA042817390731F48091D1008F7D86
:101A00008093D10014C0E091A904F091AA04E9598F
:101A1000FB4F20818091A9049091AA0401968F73B5
:101A200099279093AA048093A9042093D600FF914C
:101A3000EF919F918F913F912F910F900BBE0F903F
:101A40000FBE0F901F9018951F920F920FB60F9216
:101A500011240BB60F922F933F938F939F93EF9385
:101A6000FF9320911F0430912004809121049091D4
:101A700022042817390731F4809131018F7D80933A
:101A8000310114C0E0912104F0912204E152FC4F95
:101A90002081809121049091220401968F739927CF
:101AA000909322048093210420933601FF91EF91BB
:101AB0009F918F913F912F910F900BBE0F900FBE72
:101AC0000F901F901895CF92DF92EF92FF920F9395
:101AD0001F93CF93DF93EC016A017B014115514EB7
:101AE0006105710509F1EC89FD8981E090E008A0AC
:101AF00002C0880F991F0A94E2F7808360E079E0C2
:101B00008DE390E0A70196010E94910F89019A014F
:101B10000150110921093109369527951795079527
:101B2000980101151041A8F0EC89FD89108260E848
:101B300074E88EE190E0A70196010E94910FDA010E
:101B4000C9010197A109B109B695A7959795879500
:101B50009C01E889F9893083EA89FB89208319A2ED
:101B6000EE89FF89408181E090E09C010C8C02C0ED
:101B7000220F331F0A94E2F7242B2083EE89FF897A
:101B800040819C010D8C02C0220F331F0A94E2F7A2
:101B9000242B2083EE89FF8940819C010E8C02C09A
:101BA000220F331F0A94E2F7242B2083EE89FF894A
:101BB00020810F8C02C0880F991F0A94E2F780954C
:101BC00082238083DF91CF911F910F91FF90EF903F
:101BD000DF90CF900895CF92DF92EF92FF92EDEBDE
:101BE000F3E01382128288EEC82E83E0D82EE12C17
:101BF000F12CC482D582E682F78267EA72E07183B3
:101C000060838BEB95E09587848787E795E09787DE
:101C1000868785EC90E0918B808B84EC90E0938BB1
:101C2000828B80EC90E0958B848B81EC90E0978B9D
:101C3000868B82EC90E0918F808F86EC90E0938F82
:101C4000828F44E0448F33E0358F27E0268F95E084
:101C5000978F81E080A3EBE9F3E013821282C482C4
:101C6000D582E682F78271836083A3E3B5E0B5870E
:101C7000A487AFEEB4E0B787A687ADECB0E0B18B38
:101C8000A08BACECB0E0B38BA28BA8ECB0E0B58B32
:101C9000A48BA9ECB0E0B78BA68BAAECB0E0B18F17
:101CA000A08FAEECB0E0B38FA28F448F358F268F1C
:101CB000978F80A3E9E7F3E013821282C482D58272
:101CC000E682F78271836083ABEAB4E0B587A487CC
:101CD000A7E6B4E0B787A687A5EDB0E0B18BA08BEF
:101CE000A4EDB0E0B38BA28BA0EDB0E0B58BA48BDC
:101CF000A1EDB0E0B78BA68BA2EDB0E0B18FA08FC5
:101D0000A6EDB0E0B38FA28F448F358F268F978FCB
:101D100080A3E7E5F3E013821282C482D582E682D3
:101D2000F7827183608363E274E0758764876FED87
:101D300073E07787668765E371E0718B608B64E39E
:101D400071E0738B628B60E371E0758B648B61E390
:101D500071E0778B668B62E371E0718F608F66E371
:101D600071E0738F628F448F358F268F978F80A39A
:101D7000FF90EF90DF90CF9008950E94A3090E94FA
:101D80006D01C6E4DCE00E94AC012097E1F30E9403
:101D9000460CF9CF4F925F926F927F92AF92BF92B3
:101DA000CF92DF92EF92FF920F931F93CF93DF9327
:101DB000CDB7DEB729013A019B01AC0124193509E1
:101DC000460957098A899B89AC89BD89BC01CD0127
:101DD0006A197B098C099D090E94750FA80197015A
:101DE00024193509460957090E94B30FCA01B901E0
:101DF0006A0D7B1D8C1D9D1DDF91CF911F910F9151
:101E0000FF90EF90DF90CF90BF90AF907F906F905A
:101E10005F904F900895CF92DF92EF92FF920F93D1
:101E20001F93CF93DF936C01EB017B01E40EF51E52
:101E300000E010E0CE15DF0561F06991D601ED916B
:101E4000FC910190F081E02DC6011995080F191F32
:101E5000F1CFC801DF91CF911F910F91FF90EF90CB
:101E6000DF90CF9008956115710579F0FB01019025
:101E70000020E9F73197AF01461B570BDC01ED91CC
:101E8000FC910280F381E02D199480E090E00895A8
:101E9000DC01ED91FC910190F081E02D19940F93FC
:101EA0001F93CF93DF93EC016DE00E94480F8C01EC
:101EB0006AE0CE010E94480F800F911FDF91CF9101
:101EC0001F910F9108950F931F93CF93DF93EC0110
:101ED0000E94330F8C01CE010E944F0F800F911F83
:101EE000DF91CF911F910F910895DB018F939F9305
:101EF0000E94DA0FBF91AF91A29F800D911DA39F09
:101F0000900DB29F900D11240895991B79E004C0A3
:101F1000991F961708F0961B881F7A95C9F7809528
:101F20000895A1E21A2EAA1BBB1BFD010DC0AA1F1A
:101F3000BB1FEE1FFF1FA217B307E407F50720F032
:101F4000A21BB30BE40BF50B661F771F881F991FAD
:101F50001A9469F760957095809590959B01AC01F6
:101F6000BD01CF010895052E97FB1EF400940E9439
:101F7000CA0F57FD07D00E94910F07FC03D04EF403
:101F80000C94CA0F50954095309521953F4F4F4F77
:101F90005F4F089590958095709561957F4F8F4F15
:101FA0009F4F0895EE0FFF1F881F8BBF0790F6917C
:101FB000E02D19940E94E50FA59F900DB49F900D00
:101FC000A49F800D911D11240895A29FB001B39F7D
:101FD000C001A39F700D811D1124911DB29F700D32
:0C1FE000811D1124911D0895F894FFCF7D
:101FEC00050054657374616E646F206F73206F6CA1
:101FFC00686F73210054657374616E646F206F2079
:10200C0073696E616C20646520636172726F21006C
:10201C0054657374616E646F206F2073696E616CAC
:10202C002064652070656465737472652100546565
:10203C007374616E646F206F2062757A7A65722199
:10204C000042757A7A657220617069746F7521002F
:10205C0042757A7A6572207061726F7521004275D3
:10206C007A7A65722066756E63696F6E616E646FE5
:10207C00210054657374616E646F2061206DC3A37D
:10208C006F2100000000001A0B0B0FC30AEF0AD3DC
:04209C000A0F0B001C
:00000001FF
